:0A00DE00131211100F0E0D0C0B0A87
:100003008B128A1389148D15E4FFEFC3951550469F
:10001300AE07EEC39515503BAB12AA13A9148E82FB
:100023007583001201EDFD8F827583001201EDFCD3
:10003300D39D401C8C168E827583001201ED8F8236
:1000430075830012021A8E82758300E51612021A56
:0A0053000E80BF0F80B4E4F5802298
:10005D008B128A1389148D15E4F516AD16ED3395B3
:10006D00E0FCC3ED95157480F86C985019AB12AA8D
:10007D0013A914AF16EF3395E08F82F5831201EDBE
:07008D00F580051680D52265
:1000940078087C007D007BFF7A0079DE7E007F0A91
:1000A4001201C4750813750912750A11750B1075C0
:1000B4000C0F750D0E750E0D750F0C75100B75115B
:1000C4000A7B007A0079087D0A1200037B007A001B
:0A00D40079087D0A12005D80CA223F
:030000000200E813
:0C00E800787FE4F6D8FD758116020094C4
:1000F400E709F608DFFA8046E709F208DFFA803EEE
:1001040088828C83E709F0A3DFFA8032E309F608DA
:10011400DFFA8078E309F208DFFA807088828C8342
:10012400E309F0A3DFFA806489828A83E0A3F608F6
:10013400DFFA805889828A83E0A3F208DFFA804CD0
:1001440080D280FA80C680D4806980F280338010A7
:1001540080A680EA809A80A880DA80E280CA803310
:1001640089828A83ECFAE493A3C8C582C8CCC58388
:10017400CCF0A3C8C582C8CCC583CCDFE9DEE78058
:100184000D89828A83E493A3F608DFF9ECFAA9F0D7
:10019400EDFB2289828A83ECFAE0A3C8C582C8CC2D
:1001A400C583CCF0A3C8C582C8CCC583CCDFEADE46
:1001B400E880DB89828A83E493A3F208DFF980CCA8
:1001C40088F0ED2402B4040050C2F582EB2402B49A
:1001D400040050B823234582F582EF4E60AEEF60F1
:0901E400010EE582239001447331
:1001ED00BB010CE58229F582E5833AF583E02250C7
:1001FD0006E92582F8E622BBFE06E92582F8E22211
:0D020D00E58229F582E5833AF583E493222A
:10021A00F8BB010DE58229F582E5833AF583E8F01A
:10022A00225006E92582C8F622BBFE05E92582C8C6
:02023A00F222AE
:00000001FF
